:020000040800F2
:1000000018A300242D0400083F3800080B36000810
:100010003D3800084D0D0008D53E000800000000E6
:100020000000000000000000000000006D03000858
:100030004F0D000800000000C9030008CD3A000879
:100040004B0400084B0400084B0400084B04000854
:100050004B0400084B0400084B0400084B04000844
:100060004B0400084B0400084B0400084B04000834
:100070004B0400084B0400084B0400084B04000824
:100080004B0400084B0400084B040008710D0008E5
:10009000890D00087D0D0008950D00084B0400082F
:1000A0004B0400084B0400084B0400084B040008F4
:1000B000593C00084B0400084B0400084B0400089E
:1000C0004B0400084B0400084B0400084B040008D4
:1000D0004B0400084B0400084B0400084B040008C4
:1000E0004B0400084B040008000000004B0400080B
:1000F0004B0400084B0400084B0400084B040008A4
:100100004B0400084B0400084B0400084B04000893
:100110004B0400084B0400084B0400084B04000883
:100120004B0400084B0400084B0400084B04000873
:100130004B0400084B0400084B0400084B04000863
:1001400000000000000000000000000000000000AF
:100150004B0400084B0400084B0400084B04000843
:100160004B0400084B0400084B0400084B04000833
:100170004B0400084B0400084B040008000000007A
:100180004B0400084B0400084B0400084B04000813
:100190004B0400084B0400084B0400084B04000803
:1001A0004B0400084B0400084B040008000000004A
:1001B0004B0400084B0400084B0400084B040008E3
:1001C0004B0400084B040008000000000000000081
:1001D00000000000000000004B04000800000000C8
:1001E000000000000000000000000000000000000F
:1001F00000000000000000004B0400084B04000851
:100200004B0400084B040008000000004B040008E9
:100210004B0400084B0400084B0400084B04000882
:100220004B040008000000004B0400080000000020
:100230004B0400084B040008000000004B040008B9
:100240004B0400084B0400084B0400084B04000852
:100250004B0400084B0400084B0400084B04000842
:100260004B0400084B0400084B0400084B04000832
:100270004B0400084B0400084B0400080000000079
:100280004B0400084B0400084B0400084B04000812
:10029000000000004B0400084B04000800000000B0
:1002A000000000004B0400084B0400084B04000849
:1002B0004B0400084B0400084B040008A10D000883
:1002C000AD0D00084B0400084B04000800F002F8D4
:1002D00000F03CF80AA090E8000C82448344AAF1A4
:1002E0000107DA4501D100F031F8AFF2090EBAE8A2
:1002F0000F0013F0010F18BFFB1A43F0010318475A
:10030000485E0000685E0000103A24BF78C878C1DB
:10031000FAD8520724BF30C830C144BF04680C600B
:10032000704700000023002400250026103A28BF53
:1003300078C1FBD8520728BF30C148BF0B60704757
:100340001FB505F07FFE1FBD10B510BD00F062F9AE
:100350001146FFF7F5FF03F009FE00F080F903B442
:10036000FFF7F2FF03BC00F083F900002C4B196883
:100370000868B0E8F04F80F30988BFF36F8F4FF043
:10038000000080F3118870470000000008480068F2
:10039000006880F308884FF0000080F3148862B68C
:1003A00061B6BFF34F8FBFF36F8F00DF00BF00BF99
:1003B00008ED00E0DFF80C00016841F47001016015
:1003C000704700BF88ED00E0EFF30980BFF36F8F47
:1003D000134B1A681EF0100F08BF20ED108A20E999
:1003E000F04F106009B44FF0500080F31188BFF354
:1003F0004F8FBFF36F8F04F023FF4FF0000080F3A7
:10040000118809BC19680868B0E8F04F1EF0100F99
:1004100008BFB0EC108A80F30988BFF36F8F704774
:100420001C000024EFF30580704700000A48804755
:100430000A4880470A480047FEE7FEE7FEE7FEE776
:10044000FEE7FEE7FEE7FEE7FEE7FEE705480649B2
:10045000064A074B70470000550D0008813B000815
:10046000CD0200081873002418A300241883002468
:1004700018830024032A40F2308010F0030C00F0AF
:10048000158011F8013BBCF1020F624498BF11F8CE
:1004900001CB00F8013B38BF11F8013BA2F1040287
:1004A00098BF00F801CB38BF00F8013B11F00303FF
:1004B00000F02580083AC0F0088051F8043B083A63
:1004C00051F804CBA0E80810F5E7121D5CBF51F805
:1004D000043B40F8043BAFF30080D20724BF11F87F
:1004E000013B11F801CB48BF11F8012B24BF00F8E4
:1004F000013B00F801CB48BF00F8012B704710B555
:10050000203AC0F00B80B1E81850203AA0E818500B
:10051000B1E81850A0E81850BFF4F5AF5FEA027CCC
:1005200024BFB1E81850A0E8185044BF18C918C03B
:10053000BDE810405FEA827C24BF51F8043B40F8DC
:10054000043B08BF7047D20728BF31F8023B48BFC1
:1005500011F8012B28BF20F8023B48BF00F8012BFF
:10056000704702F0FF0343EA032242EA024200F02E
:100570002CB84FF0000200B5134694469646203939
:1005800022BFA0E80C50A0E80C50B1F12001BFF44C
:10059000F7AF090728BFA0E80C5048BF0CC05DF8B2
:1005A00004EB890028BF40F8042B08BF704748BF00
:1005B00020F8022B11F0804F18BF00F8012B704774
:1005C0007047704770474FF000020429C0F0128056
:1005D00010F0030C3FF4CFAFCCF1040CBCF1020FD0
:1005E00018BF00F8012BA8BF20F8022BA1EB0C01CB
:1005F000FFF7C1BF5FEAC17C24BF00F8012B00F800
:10060000012B48BF00F8012B7047000000487047DD
:10061000B47200247546FFF7F9FFAE46050069463F
:10062000534620F00700854618B020B5FFF70EFFAF
:10063000BDE820404FF000064FF000074FF00008E3
:100640004FF0000B21F00701AC46ACE8C009ACE864
:10065000C009ACE8C009ACE8C0098D46704710B5C8
:100660000446AFF300802046BDE81040FFF777BE98
:1006700001491820ABBEFEE72600020070470000CB
:100680002DE9F04716008846074600D10A261F4C80
:100690006421A06803F0C8FD18B16FF00400BDE844
:1006A000F08760684FF0FF390BE00178B94207D15D
:1006B0004268424504D1A06803F013FE4846EEE7C5
:1006C00000690028F1D1142000F03EFB050012D093
:1006D00000223046542103F047FDA86088B12F70F6
:1006E000C5F804802E73606828616560A06803F017
:1006F000F8FD0020D3E7A06803F0F3FD6FF00100E0
:10070000CDE7284600F01EFBD5E700009C00002442
:1007100070470000074A526808E01378834204D10A
:1007200053688B4201D1906870471269002AF4D156
:10073000002070479C000024D0E901014FF0804266
:10074000B1F1005F03D0904207D101207047904281
:1007500001D103207047022070470020704700003D
:10076000032804D228B1012805D0022805D0002092
:1007700070470348704703487047034870470000BC
:10078000B000002450010024F00100242DE9F041C4
:10079000164C0746984615460E46207848B15DB17E
:1007A000A068642103F040FD48B16FF00400BDE88B
:1007B000F0816FF00200FAE76FF00100F7E73146D1
:1007C0003846FFF7A7FF0646A06803F08AFD56B13A
:1007D000002243462946304603F094FC0028E6D028
:1007E0004FF0FF30E3E76FF00300E0E79C000024E8
:1007F000F0B56A4E89B0307818B16FF0020009B0D8
:10080000F0BD67486021FFF7B4FE654A002420462A
:100810006032C1B2032908D240F29113594302EB6E
:10082000C101C1F8804CC1F8844C401C0328F0DBA6
:100830005C48F060002003F020FD0028B0607CD010
:100840000127377002940225019401A95648CDE989
:10085000047403950694079400F062FC0222524847
:1008600000231146009400F09AFC039501A9CDE9FC
:1008700001474D48CDE904740694079400F050FCFC
:100880000222494800231146009400F088FCCDE97B
:100890000145464801A9CDE90454039506940794FF
:1008A00000F03EFC0222414800231146009400F073
:1008B00076FC03200194CDE902053C4801A9CDE96D
:1008C00004540694079400F02BFC022237480023BE
:1008D0001146009400F063FC04200194CDE9020568
:1008E000334801A9CDE904540694079400F018FC9C
:1008F00002222F4800231146009400F050FC0520EE
:100900000194CDE902052A4801A9CDE904540694D1
:10091000079400F005FC02222548002311460094AC
:1009200000F03DFC234900221F4800F081FB214CD0
:1009300000221E480F34214600E02CE000F078FB36
:100940001B480022214600F073FB184801F014F9FF
:10095000174801F011F9184A0321002000F03AF875
:100960000021164A084600F035F8154A05210120F5
:1009700000F030F8114A0021012000F02BF8104A55
:100980000521022000F026F80C4A0021022000F088
:1009900021F8002033E74FF0FF3030E79C000024BF
:1009A000B04B002411070008B000002450010024BF
:1009B000F001002401100200250A0008A50C00081F
:1009C000C10A0008024AD268002A00D010477047C6
:1009D0009C0000240C4B1B7843B152B103284FF00C
:1009E000FF3301D2082907D3184670476FF0020081
:1009F00070476FF001007047044B03EB401040F864
:100A000021200020704700009C000024B04B0024EF
:100A1000034B1B780BB1FFF733BE6FF0020070473A
:100A20009C0000242DE9F0430024AFB0E0B2FFF7B2
:100A300097FE06003BD034E0402130461FAB15AA9C
:100A400000F0E6FB98BB16980028159835D020F0EA
:100A5000604515A8FFF770FE804601462846FFF75F
:100A6000B1FF81464946E0B2FFF754FE070018D0B7
:100A70008DF80080CDE901591898C0B28DF80C00AE
:100A8000402802D940208DF80C00C2B21FA90DF1F8
:100A90000D00FFF7EFFC002369461A46384603F0C5
:100AA0008FFB4021304600F0A7FB0028C4D1641C16
:100AB000032CBBDB2FB0BDE8F083C0F30A05C8E709
:100AC0002DE9F0430024AFB0E0B2FFF749FE060085
:100AD0003BD034E0412130461FAB15AA00F098FB13
:100AE00098BB16980028159835D020F0604515A8B9
:100AF000FFF722FE804601462846FFF763FF814646
:100B00004946E0B2FFF706FE070018D08DF80080D6
:100B1000CDE901591898C0B28DF80C00402802D9CF
:100B200040208DF80C00C2B21FA90DF10D00FFF797
:100B3000A1FC002369461A46384603F041FB4121D7
:100B4000304600F059FB0028C4D1641C032CBBDBE9
:100B50002FB0BDE8F083C0F30A05C8E72DE9F04FD8
:100B6000DFF838A199B00646984615460F46229CF4
:100B70009AF8000048B1032E4FF0FF3B7DD2B8F148
:100B8000000F6FF0010105D008E06FF0020019B00E
:100B9000BDE8F08F022F01D0032F18D1402C6CD864
:100BA0003046FFF7DDFD5FEA000910D0642168469A
:100BB000FFF7DFFC4FF000005FB1012F4FF08041E5
:100BC0000BD04A10022F0CD0032F56D10DE008464F
:100BD000DDE7CDE9005002900AE00095CDE9011073
:100BE00006E00095CDE9010202E00095CDE9011291
:100BF0000121089105AD04904A05CB0585E80D005B
:100C0000082C01D808200CE0182C01D80C2008E092
:100C1000202C01D20D2004E0302C01D20E2000E067
:100C20000F200390B8F1000009AD05D024B1224691
:100C300001462846FFF71EFC484600F007FCCAF8AC
:100C40001000484600F002FC30B12A46694648468A
:100C500000F032FA00289AD040F29110104A69460A
:100C600016FB00F002EBC004D4F8800CD4F8842CFE
:100C7000401C00F01F05AA4201D1584687E7D4F86E
:100C8000800C00EBC00202EB0010642204EB800039
:100C9000FFF735FCC4F8805C002078E79C00002456
:100CA000104C00242DE9F041DFF894800025A4B019
:100CB000ECB22046FFF754FD07003AD019A9384698
:100CC00000F06CFB0028F9D020E0032C684630D2FD
:100CD000D6F8801CD6F8842C91422AD0D6F8841CF1
:100CE00001EBC10202EB0111642206EB8101FFF767
:100CF00006FCD6F8840C401C00F01F00C6F8840CDB
:100D000009AA6946384600F0D7F990B9032C10D2E9
:100D100040F2911204FB02F108EBC106D6F8800CF8
:100D2000D6F8841C884204D0384600F08FFB002897
:100D3000CBD16D1C032DBBDB24B0BDE8F0810000DE
:100D4000104C002404F04EB803F028BFFEE77047B3
:100D500072B6FEE7054805490839026842F002020A
:100D6000026008688004FCD5704700000C480258F7
:100D7000014800F073BB0000B0000024014800F0FF
:100D80006DBB0000B0000024014800F067BB00000C
:100D900050010024014800F061BB00005001002414
:100DA000014800F05BBB0000F0010024014800F0A6
:100DB00055BB0000F0010024F0B503684FF6FC714C
:100DC0006D4C426BD3F884508D4345EA8205C3F8DD
:100DD0008450036853F8845F068F25F47F0545EA45
:100DE00006451D60836B654D9F180268D2F88830F8
:100DF0008B4343EA8703C2F88830026852F8883F81
:100E0000868F23F4FE0343EA06431360066856F810
:100E1000A03FC26B8B4307EB420243EA820333607D
:100E2000076857F8A03FB0F8406023F4FE0343EA98
:100E300006433B60D0E9103603FB06220368D3F873
:100E4000B0608E4346EA8206C3F8B0600368B0F82B
:100E50004860D3F8B07027F4FE0747EA0646C3F8A7
:100E6000B060D0E91267036806FB0722D3F8AC60D4
:100E70008E4346EA8206C3F8AC60D0E91467036883
:100E800006FB0722D3F8F0608E4346EA8206C3F8D9
:100E9000F0600368B0F85860D3F8F07027F47C175E
:100EA00047EA0646C3F8F0600368876D53F8C06FE1
:100EB00002EB47028E4346EA820119600168B0F8EE
:100EC0005C20D1F8C03023F47C1343EA0242C1F81D
:100ED000C020016890F86020D1F8C03023F07C5326
:100EE00043EA0262C1F8C020416B04EB8101C16694
:100EF000826B01EB82020267C36B02EBC3024267A3
:100F0000D0E91034634302EB83028267D0E91234E4
:100F1000634302EB8302C267D0E91434634302EBFC
:100F20008302C0F88020836D02EBC303C0F88430D5
:100F3000C46D826E544303EB8403C0F88830046EA2
:100F4000544303EB8402C0F89020AA420AD9D0F897
:100F50009C20032142F02002C0F89C2080F89810C9
:100F60000120F0BD002200E004C1D0F890308B4297
:100F7000FAD80020F0BD000000AC0040FCD30040D7
:100F8000F0B58E680C69D1E9005744EA0604DFB178
:100F900045F080452C43866ED1E906C54F695E4316
:100FA00091F8203045EA0C05B1F80CC0D0F884E087
:100FB000002047EA0363104F1D430EEB860345EA0A
:100FC0000C45E3E8024511E044EA8544E3E71418E0
:100FD000155CA67894F803C094F801E0360445EA5D
:100FE0000C6446EA0E252C43001D10C3CC683C5D02
:100FF0008442ECD8F0BD00007460000878B100684D
:101000000849884201D1002070470749884201D130
:10101000012070470549884201D102207047042011
:101020007047000000A0004000A4004000D4004031
:1010300010B590F89830012B09D0022B07D0D0F8CA
:101040009C1041F00201C0F89C10012010BD036803
:101050009C6D0C4203D1DC6D44F0010404E09C6DF6
:1010600031EA04041FD00324DC658B0505D5036831
:10107000D3F8E0401443C3F8E0404B0505D50368BE
:10108000D3F8E4401443C3F8E4400068084A01EA96
:101090000203446D074A1C434465106840EA91709E
:1010A0001060002010BDDC6D44F00204DCE700009D
:1010B000FFFFCF3F14A8004070B5044690F8980099
:1010C000022804D0D4F89C0040F008000DE020680D
:1010D000D0F8C03013F07C5F0BD0D0F8C4309B0246
:1010E0000CD5D4F89C0040F40070C4F89C0001209A
:1010F00070BDD4F89C0040F02000F6E7D0F8C400A2
:10110000C0F3044520462B46FFF73AFF2168012033
:10111000A840C1F8D000C4F89400002070BD70470A
:1011200070B590F89820012A09D0022A07D0D0F88B
:101130009C1041F00201C0F89C10012070BD0B68AA
:10114000CA6883B10B69072A43EA427325D00C7A37
:101150004A6942EA84724968006F00EBC100C0E945
:101160000032002070BD072A0DD00C7AD6060D8AF9
:101170004B6943EA847246EA0543C06E49681A43E4
:1011800040F82120EDE70B8A4FF06055D1E90624A5
:1011900042EA034245EA0423EFE78A69DBE730B518
:1011A00090F89850039C012D07D0D0F89C1041F086
:1011B0000401C0F89C10012030BD0D01016845EA12
:1011C000820040EA43002043C1F88000002030BD87
:1011D00010B5FFF713FF042808D0054901EB4010B4
:1011E000C069002802D0BDE81040004710BD0000D3
:1011F000B04B0024704700000068402905D0D0F8AB
:10120000B40000BF00F07F007047D0F8A400F9E7F9
:10121000F0B590F898500024022D04D0D0F89C101E
:1012200041F0080129E0402905D0412929D0056D68
:101230008D4219D942E00568D5F8A06016F4FE0F7A
:1012400012D0D5F8A460760613D0D5F8A460F601C4
:1012500005D5D5F8A06016F0004F00D50124D5F8CB
:10126000A470466F456C24E0D0F89C1041F020013A
:1012700003E0D0F89C1041F48071C0F89C1001206C
:10128000F0BD0568D5F8B06016F4FE0FECD0D5F8C7
:10129000B4607606EDD0D5F8B460F60105D5D5F882
:1012A000B06016F0004F00D50124D5F8B470866FF9
:1012B000C56CC7F305273C44654302E0456DC66F26
:1012C0004D4306EB85052E6816F0804656602E6865
:1012D00036D026F060461660D5F800C000262E4FA6
:1012E0000CF0005CC2F808C0D5F800C00CF0004C4F
:1012F000C2F810C0B5F804C01FFA8CFCC2F81CC0BC
:10130000D5F804C0CCF3034CC2F80CC0D5F804C027
:101310000CF4801CC2F814C0D5F804C00CF4001CF6
:10132000C2F818C0D5F804C0CCF3066CC2F820C0CF
:10133000D5F804C008354FEADC7CC2F824C008E0C8
:10134000C6F38A46C7E700BF15F806C003F806C013
:10135000761CD2F80CC017F80CC0B445F4D840295C
:101360000AD041290CD020294FF001020CD200688C
:101370008A40C0F898200DE00068C0F8A84009E055
:101380000068C0F8B84005E0006801F01F018A401D
:10139000C0F89C200020F0BD7460000810B590F8E3
:1013A0009820022A04D0D0F89C1041F0080146E0B1
:1013B0000268D2F8F03013F47C1F37D0D2F8F43042
:1013C0009B0638D0D2F8F430D0F88020C3F3042341
:1013D00002EBC302146814F080444C60146832D0ED
:1013E00024F060440C60146804F000548C601468AD
:1013F00004F000440C619488A4B2CC615468C4F336
:101400000344CC60546804F480144C61546804F4C0
:1014100000148C61546804F440044C625268120E4B
:101420000A620068C0F8F830002010BDD0F89C10A7
:1014300041F0200103E0D0F89C1041F48071C0F825
:101440009C10012010BDC4F38A44CBE70068D0F89B
:10145000C40000F03F007047704700002DE9FF5FB7
:10146000DFF80CB304460BF10401DBF8000025683B
:101470000F68AA468007D5F85090696DD5F850805E
:101480006E6D2A6DD5F854C02B6D00EA8770009000
:1014900009F470496F6D286D01EA09010191DAF8CC
:1014A0005410DAF85490DAF8505008F00F0806EAB1
:1014B0000806029602F0F00203F071536FEA090683
:1014C0001F4000F060700CEA020CCDF80CC0F20571
:1014D00001EA00090CD4E843C00509D400214FF407
:1014E0008073CAF85030CBF800102046FFF7B4FFE5
:1014F000700512D4E84340050FD4206800234FF450
:101500008068D0F8DC20D0F8E410C0F85080CBF828
:1015100000301140204600F04FFBDFF858A2009841
:1015200050B12268830F00EA0A001065CBF8003042
:1015300020460099FFF7F3FD019850B12268830F10
:1015400000EA0A001065CBF800302046019900F04F
:1015500057FB029850B12268830F00EA0A00106519
:10156000CBF800302046029900F0E2FA039850B11F
:101570002268830F00EA0A001065CBF8003020468D
:10158000039900F0E7FA30050CD4E843000509D4CC
:10159000236800204FF400621A65CBF80000204653
:1015A00000F040FBB00512D4E84380050FD420685A
:1015B00000234FF40078D0F8D820D0F8E010C0F81D
:1015C0005080CBF800301140204600F007FB30037C
:1015D0000CD4E843000309D4236800204FF4002210
:1015E0001A65CBF80000204600F0A0FAF0030CD4F6
:1015F000E843C00309D4236800204FF480321A6501
:10160000CBF80000204600F0D5FA70030CD4E84374
:10161000400309D4226800204FF480231365CBF8DF
:101620000000204600F0C5FAB0030FD4E843800361
:101630000CD4236800204FF400321A65CBF8000068
:10164000D4F89C0040F08000C4F89C00B9F1000F71
:101650000BD022684FEA997309EA0A001065CBF8AB
:10166000003049462046FFF7C5FD5FB12268BB0F39
:1016700007EA0A001065CBF80030D4F89C00384324
:10168000C4F89C003C492068884268D16068814663
:101690008068800763D0D9F82060D9F82410D9F881
:1016A0002080D9F82400D9F820C0D9F82470D9F8BE
:1016B0002030D9F82450D9F8202003F4FC4306F058
:1016C0000F0AD9F824601D40D9F824B008F030087A
:1016D0000CF4C07C02F4F02211EA0A0100EA0808C6
:1016E00007EA0C0706EA0206D9F820A004D0C9F8D8
:1016F0002010204600F05AFAB8F1000005D06168C9
:1017000008624146204600F053FA6FEA0B0040069B
:101710000ED46FEA0A0040060AD460684021C36B09
:10172000C26B01622046190C02F03F0200F03FFA42
:101730002FB1606807623946204600F036FA35B1AD
:1017400060680562D4F89C002843C4F89C0036B158
:1017500060680662D4F89C003043C4F89C00D4F85A
:101760009C00002802D02046FFF732FDBDE8FF9F15
:1017700010A80040FFFFCF3F00A000402DE9F0413E
:1017800094B08D494C2204466846FEF7B8FE64B119
:101790008A4D2068A84202D100F58070606094F8FC
:1017A00098004FF0000820B108E0012014B0BDE817
:1017B000F081204684F8998000F002F92068816960
:1017C00021F01001816100F043FB0327064604E08D
:1017D00000F03EFB801B0A2811D8206880690007B2
:1017E000F6D42068816941F00101816100F030FB8D
:1017F00006460DE000F02CFB801B0A2808D9D4F81F
:101800009C0040F00100C4F89C0084F89870CCE77C
:1018100020688069C007EDD02068816941F002012D
:101820008161207C01282068816937D041F0400126
:101830008161607C01282068816932D021F4804177
:101840008161A07C0128206881692DD041F48051FC
:1018500081612068A268816921F44071114381612E
:101860002068816921F0A40181612068016921F06B
:1018700010010161E068012819D010B302281BD0C3
:101880002068816941F0800181612068016941F02F
:1018900010010161E06803280ED012E021F0400140
:1018A000C6E741F48041CBE721F48051D0E72068BE
:1018B000816941F0040103E02068816941F0200161
:1018C0008161207E6FF0FF02D4E90773A68A1102BE
:1018D000400602EB0727A0F10070384327685B1E23
:1018E000184301EB06463043F861A068B0F5407F2D
:1018F00011D104F12800A68C6FF00F0C89C801EB00
:101900000641401E02EB0322104322680CEB071332
:1019100018430843D060206E30B12068626ED0F862
:10192000C0101143C0F8C010D4E917126846D14264
:1019300009D02168A36E51F8C82F50F8233022F047
:1019400007021A430A60216C49B12168626C51F8A0
:10195000BC3F50F8226023F0070232430A60A16CBA
:1019600051B12168E36C51F8BC2F50F8233022F0BC
:10197000700242EA03120A60216D51B12168626D62
:1019800051F8BC3F50F8220023F4E06242EA002004
:1019900008602068A84204D16068816821F00301D2
:1019A0008160C4F894800121C4F89C8084F8981068
:1019B0002046FFF701FAF9E68460000800A0004025
:1019C000F0B587B0054614216846FEF7D2FD514EAA
:1019D00000244F4B02272D684FF0090CDFF838E147
:1019E0000C3B31684A4A75454C4801F101012AD146
:1019F0000129316007D1116841F4807111601168CB
:101A000001F480710591196841F0080119601968A5
:101A100001F00801059103210091CDE90174CDE9A0
:101A2000034C694600F000F900220521132000F064
:101A3000FFFA132000F0EEFA00220521152000F035
:101A4000F7FA15202EE0DFF8D8E075452ED10129F0
:101A5000316007D1106840F480701060106800F4A5
:101A600080700590186840F0020018601868694698
:101A700000F00200059060200090CDE90174294833
:101A8000CDE9034C00F0D0F800220521142000F02D
:101A9000CFFA142000F0BEFA00220521162000F033
:101AA000C7FA162000F0B6FA07B0F0BDDFF878C02C
:101AB0006545F9D10129316007D1116841F4807180
:101AC0001160116801F480710591196841F00801F5
:101AD00019601968052201F0080105914FF4405181
:101AE0000091CDE90174CDE90342694600F09CF80C
:101AF000002205219F2000F09BFA9F2000F08AFA27
:101B000000220521A02000F093FAA020CAE70000DF
:101B1000EC4402580400002400A00040000C0258CD
:101B200000A400400004025800D4004070470000A8
:101B300010B5FFF763FA042808D0054901EB4010FF
:101B4000C068002802D0BDE81040004710BD00006A
:101B5000B04B002410B5FFF751FA042808D005490E
:101B600001EB40104069002802D0BDE8104000475A
:101B700010BD0000B04B002490F89810012907D048
:101B8000D0F89C1041F00401C0F89C10012070476F
:101B9000022180F89810002201688B6923F001036C
:101BA0008B61C0F89C2010467047704770477047A3
:101BB000704770477047000010B5FFF71FFA042800
:101BC00008D0054901EB40108068002802D0BDE82C
:101BD0001040004710BD0000B04B002410B5FFF7C7
:101BE0000DFA042808D0054901EB40104068002890
:101BF00002D0BDE81040004710BD0000B04B0024EB
:101C000010B5FFF7FBF9042808D0054901EB401097
:101C10000068002802D0BDE81040004710BD000059
:101C2000B04B0024704700002DE9F84F03247A4D93
:101C300000234FF001094FF0B04B4FF00F0AE4E0E2
:101C400009FA03F6324078D00F7907F00307012F25
:101C500001D0022F1AD187684FEA430ED1F80CC089
:101C600004FA0EF827EA08070CFA0EFC4CEA070CF7
:101C7000C0F808C0476891F804C0B743CCF3001C13
:101C80000CFA03FC4CEA070CC0F804C00E79F643CA
:101C9000B6070BD0C6684FEA43088F6804FA08FC01
:101CA00026EA0C0607FA08F73743C7600E7906F0F4
:101CB0000306022E12D1DE080F694FEA437C00EBC7
:101CC0008606B646366A4FEADC6C0AFA0CF807FA62
:101CD0000CF726EA08063743CEF820700F7906681D
:101CE0004FEA430807F0030704FA08FC07FA08F76D
:101CF00026EA0C06374307604E6816F4403F1CD0B6
:101D0000464E376847F00207376036689F0706F08F
:101D10000206009623F0030606F1B046B6463F0FD2
:101D2000D6F80864DFF8F8800AFA07FC404526EA8E
:101D30000C0603D14FF0000C3AE065E0DFF8E4C098
:101D4000604502D14FF0010C32E0DFF8DCC06045A5
:101D500002D14FF0020C2BE0DFF8D0C0604502D179
:101D60004FF0030C24E0DFF8C8C0604502D14FF00B
:101D7000040C1DE0DFF8BCC0604502D14FF0050C3B
:101D800016E0DFF8B4C0604502D14FF0060C0FE05A
:101D9000DFF8A8C0604502D14FF0070C08E0DFF87B
:101DA000A0C0604502D14FF0090C01E04FF00A0CD1
:101DB0000CFA07FC4CEA060CCEF808C44F68DBF8B6
:101DC0000060FF0226EA020600D516435F46CBF804
:101DD0000060D1F804C0DBF804605FEA8C2C26EACE
:101DE000020600D516437E606E684F6826EA02063A
:101DF000BF0300D516436E602E684F6826EA0206C0
:101E0000FF0300D516432E605B1C0A6832FA03F606
:101E10007FF416AFBDE8F88F80000058F4440258F4
:101E2000000002580004025800080258000C025832
:101E3000001002580014025800180258001C0258E2
:101E4000002402580AB1816170470904FBE70000D1
:101E5000014880687047000008000024024881683B
:101E6000027811448160704708000024032010B5F7
:101E700000F0FEF800F066FF0F4A1049146813687E
:101E8000C4F3032203F00F038A5CC95C02F01F0253
:101E900001F01F01D0400A4A20FA01F111600949FE
:101EA00008600F2000F010F808B1012010BD00F00C
:101EB0009FF8002010BD000018440258D0600008B0
:101EC000180000241400002410B5102804468AB01D
:101ED0002DD2002201461C2000F0AAF81C2000F0A0
:101EE00099F8184804601848016841F00101016040
:101EF000006809A900F001000890684600F0C0FEE3
:101F00000598B8B100F00CFF40001049002240F2E3
:101F1000E733B0FBF1F10E484FF080440460C0E9B4
:101F20000332491EC0E9011201F03EFA28B1012036
:101F30000AB010BD00F0F4FEE7E7054801F066FACC
:101F4000F6E700000C000024E844025840420F006D
:101F500090020024154BF0B5083B427813491A60F3
:101F60000B680A1F23F001030B6043681360057BB5
:101F7000C67A827A437B2D07847B45EA0665C77B58
:101F800090F809C0067A90F800E045EAC24040EABD
:101F9000834040EA444040EA074040EA0C2040EADF
:101FA000460040EA0E000860F0BD0000A0ED00E031
:101FB000BFF35F8F044800210368034A23F4803392
:101FC000036070321160704724ED00E0074A40F072
:101FD0000100064970321060086840F480300860E3
:101FE000BFF34F8FBFF36F8F7047000024ED00E009
:101FF000074882B0016841F00201016000680022D8
:102000000F2100F002000090901E02B000F010B806
:10201000F4440258002809DB410900F01F0289003E
:10202000012001F1E0219040C1F80001704700005B
:102030000E4BF0B41B680D46C3F30223C3F1070631
:10204000042E00D90426191D072901D2002300E01F
:10205000DB1E012404FA06F19C40491E2940641E3F
:10206000994014402143F0BC01F035BF0CED00E075
:10207000064900F0070210B54FF6FF040868044B4C
:10208000204040EA02201843086010BD0CED00E03B
:102090000000FA05134970B50A68D243520705D506
:1020A000096801F00701814213D118E00A6822F0A3
:1020B000070202430A60FFF7CBFE0A4D4FF47A761F
:1020C0000446083D07E000BFFFF7C2FE001BB04218
:1020D00001D9012070BD2868C0438004F4D40020D9
:1020E00070BD00000C4802582DE9FE4F0546DFF890
:1020F00000A450F8081B0024FD4FC943019005F1CE
:10210000280026460AF1240A009008011DD4686EB2
:1021100050B1B0F5801F0CD0B0F5001F0ED0B0F557
:10212000401F1ED001240FE0386840F400303860B2
:1021300017E00198022101F0A5FB03E000980221BD
:1021400001F030FC04000CD026462888C043C005AE
:1021500023D4A86D05281ED2DFE800F00C11161B51
:102160001B006A6EDAF8001021F440111143CAF81E
:102170000010EAE7386840F40030386009E0019860
:10218000002101F07FFB03E00098002101F00AFC30
:102190000446C4B100E0012426462888DFF85083B5
:1021A000C04308F12C0840052FD4D5F8A400B0F5A1
:1021B000C00F28D010DCB8B1B0F5001F19D0B0F5B1
:1021C000800F0FD11AE0AA6DDAF8001021F0070194
:1021D0001143CAF80010E0E7B0F5000F13D0B0F5D6
:1021E000200F10D001240FE0386840F40030386030
:1021F00009E00198002101F045FB03E0009800216F
:1022000001F0D0FB044694B126462888C04300055F
:1022100030D4D5F8A800B0F1407F29D011DCC0B18E
:10222000B0F1807F1AD0B0F1007F10D11BE0D5F85B
:10223000A420D8F8001021F460011143C8F8001060
:10224000E3E7B0F1806F13D0B0F1A06F10D001249C
:102250000FE0386840F40030386009E00198002150
:1022600001F010FB03E00098002101F09BFB044605
:1022700094B126462868DFF878B2C0430BF1200BF2
:1022800080011FD4E86CD8B110280FD0202812D0BC
:10229000302815D0012414E0D5F8A820D8F8001073
:1022A00021F0E0611143C8F80010E3E7386840F41A
:1022B0000030386004E00198022101F0E3FA04469E
:1022C00074B126462888C043C0042BD4E86DB0F50D
:1022D000005F20D00DDCA0B1B0F5805F0FD115E01C
:1022E000EA6CDBF8001021F030011143CBF800104C
:1022F000E8E7B0F5405F13D0B0F5804F10D001246F
:102300000FE0386840F40030386009E0019800219F
:1023100001F0B8FA03E00098002101F043FB044605
:102320008CB126462888C043800429D4286EB0F595
:10233000403F23D010DC08B3B0F5803F14D0B0F597
:10234000003F0FD115E0EA6DDAF8001021F4E0410A
:102350001143CAF80010E5E7B0F5802F0ED0B0F5B4
:10236000A02F0BD001240AE00198012101F08AFA84
:1023700003E00098012101F015FB044694B12646C4
:102380002888C04340042AD4D5F8AC00B0F1405F9F
:1023900023D010DC08B3B0F1805F14D0B0F1005F3F
:1023A0000FD115E02A6EDAF8001021F4E021114374
:1023B000CAF80010E4E7B0F1804F0ED0B0F1A04FA2
:1023C0000BD001240AE00198012101F05BFA03E03F
:1023D0000098012101F0E6FA044674B126462888E7
:1023E000C04300041FD4E86ED8B1B0F1805F0ED0B6
:1023F000B0F1005F10D0012414E0D5F8AC20D8F87B
:10240000001021F0E0411143C8F80010E7E73868F8
:1024100040F40030386004E00198012101F032FA04
:10242000044674B126462868C043C0011ED4A86C77
:10243000D0B101280ED0022811D0032814D00124D5
:1024400013E0EA6EDAF8001021F040511143CAF8A7
:102450000010E8E7386840F40030386004E0019884
:10246000022101F00FFA04466CB126462868C043E9
:10247000400255D41F48016841F480710160FFF7A4
:10248000E7FC81460EE0AA6CDBF8001021F00301A6
:102490001143CBF80010E9E7FFF7DAFCA0EB0900E5
:1024A00064283BD813480068C005F5D5BCBBDFF8ED
:1024B0004090B5F8B01009F14409D9F8000001F4D2
:1024C000407100F44070884211D0D9F80010D9F85A
:1024D000002021F4407142F48032C9F80020D9F87C
:1024E000002022F48032C9F80020C9F8001003E06F
:1024F0002C44025800480258D5F8B000B0F5807F4F
:1025000019D1FFF7A5FC029011E000BFFFF7A0FC76
:102510000299411A41F28830814208D903242646A3
:102520002878DFF81494C043C00721D03CE0D9F8E4
:1025300000008007EAD5D5F8B010C1F301200328C8
:10254000FE480DD0016821F47C510160B5F8B0203F
:10255000D9F80010C2F30B021143C9F80010DFE7ED
:10256000F74A036802EA111223F47C511143ECE7A5
:10257000A86F182816D005DCA0B1082808D01028AC
:1025800004D10AE020280DD028280BD001240AE02D
:102590000198012101F076F903E00098012101F092
:1025A00001FA044664B126462878C04380071ED449
:1025B000686F062819D2DFE800F0160C11161616FF
:1025C000AA6FD9F8001021F038011143C9F80010A2
:1025D000EAE70198012101F055F903E00098012193
:1025E00001F0E0F904467CB100E001242646287899
:1025F000C04340071FD4D5F89000062819D2DFE861
:1026000000F0160C111616166A6FD9F8001021F09A
:1026100007011143C9F80010E9E70198012101F011
:1026200031F903E00098012101F0BCF90446A4B19E
:1026300000E0012426462878C04380062BD4D5F834
:102640008C00B0F1405F24D011DC10B3B0F1805F9A
:1026500015D0B0F1005F10D116E0D5F89020D8F871
:10266000001021F007011143C8F80010E3E7B0F1B2
:10267000804F0ED0B0F1A04F0BD001240AE001989A
:10268000002101F0FFF803E00098022101F08AF92F
:10269000044694B126462878C04340062BD4D5F88A
:1026A0009800B0F5406F24D011DC10B3B0F5806F06
:1026B00015D0B0F5006F10D116E0D5F88C20D9F800
:1026C000001021F0E0411143C9F80010E3E7B0F534
:1026D000805F0ED0B0F5A05F0BD001240AE0019816
:1026E000002101F0CFF803E00098022101F05AF92F
:1026F000044694B126462878C04300062BD4D5F86A
:102700009C00B0F5C04F24D011DC10B3B0F5005FD1
:1027100015D0B0F5804F10D116E0D5F89820D8F834
:10272000001021F4E0511143C8F80010E3E7B0F5C0
:10273000004F0ED0B0F5204F0BD001240AE00198D5
:10274000002101F09FF803E00098022101F02AF92E
:10275000044654B126462878C04300071ED4D5F855
:102760008000B0F5805F0AD00FE0D5F89C20D8F843
:10277000001021F460411143C8F80010EBE7009805
:10278000022101F00FF900B10126D5F88020D9F817
:10279000001021F440511143C9F800102878C043BB
:1027A000C00613D4D5F89400B0F5807F05D1009809
:1027B000022101F0F7F800B10126D5F89420D8F8ED
:1027C000001021F440711143C8F800102868C0437C
:1027D000000316D4D5F8A00038B1B0F5803F09D079
:1027E000B0F5003F0BD001240AE00198002101F070
:1027F00049F803E00098022101F0D4F804468CB1B6
:1028000026462868C043400322D4D5F88400B0F59A
:10281000801F11D0B0F5001F13D0B0F5401F15D0A8
:10282000012414E0D5F8A020D8F8001021F440319C
:102830001143C8F80010E4E7386840F4003038600D
:1028400004E00098012101F0ADF804465CB1264691
:102850002868C043C0031CD4286D70B1B0F5803F18
:1028600010D0012414E0D5F88420D9F8001021F408
:1028700040111143C9F80010EAE7386840F400300D
:10288000386004E00198022100F0FCFF0446DCB14E
:1028900026462868C043800005D40098022101F034
:1028A00081F800B101262868C04380031BD4E86F7B
:1028B000B8B1B0F5807F10D0B0F5007F11D0B0F581
:1028C000407F0ED001240DE02A6DDBF8001021F4CA
:1028D00080311143CBF80010DBE7386840F400305A
:1028E00038607CB326462868C043C00207D42A6FEC
:1028F000DAF8001021F000411143CAF800102868EE
:10290000C043800207D4AA6EDAF8001021F080716B
:102910001143CAF800102868C043400009D4074892
:10292000016821F4004101600168D5F8B420114329
:1029300001602868C04306E054440258104402581D
:10294000CFFFFF001DE007D46A6DDBF8001021F017
:1029500040511143CBF800102868C043000208D44E
:10296000D5F88820D9F8001021F440011143C9F8A6
:10297000001028790024C04300F00100204309D052
:102980000EE0EA6FD9F8001021F440711143C9F844
:102990000010A8E70198002100F074FF00B106467E
:1029A0002879C04300F00200204305D1019801219D
:1029B00000F068FF00B106462879C04300F004002B
:1029C000204305D10198022100F05CFF00B10646CA
:1029D0002879C04300F00800204305D10098002169
:1029E00000F0E0FF00B106462879C04300F0100077
:1029F000204305D10098012100F0D4FF00B1064624
:102A00002879C04300F02000044304D1009802213B
:102A100000F0C8FF00B916B10120BDE8FE8F00200C
:102A2000FBE700002DE9F05F04000F467ED0DFF8E1
:102A30003882D8F8000000F00F00B8420CD2D8F865
:102A4000001021F00F013943C8F80010D8F8000039
:102A500000F00F00B84269D12078844D40070AD5B4
:102A60002069296801F07001884204D9296821F0A1
:102A700070010143296020787C4E361D00070AD57D
:102A80006069316801F07001884204D9316821F031
:102A90007001014331602078C0060AD5A069316811
:102AA00001F4E061884204D9316821F4E061014316
:102AB00031602078DFF8B4B180060BF1080B0CD53B
:102AC000E1695846DBF8002002F07002914204D917
:102AD000026822F070020A430260207880070AD55B
:102AE000E068296801F00F01884204D9296821F0C3
:102AF0000F01014329602078C0073ED05B49A268DE
:102B00002868183920F47060104328606068022833
:102B100018D0032819D00968012819D049070029BD
:102B20004ADADFF848A1AAF1080A00E044E0DAF83E
:102B3000002022F007020243CAF80020FFF788F9BC
:102B4000814612E009688903E9E709688901E6E737
:102B5000C905E4E7FFF77CF9A0EB090141F28830F1
:102B6000814202D90320BDE8F09F6168DAF80000D5
:102B700000F03800B0EBC10FECD1207880070AD507
:102B8000E068296801F00F01884204D2296821F029
:102B90000F0101432960D8F80010404601F00F01F1
:102BA000B9420BD9016821F00F0139430160006877
:102BB00000F00F00B84201D00120D4E72078400790
:102BC0000AD52069296801F07001884204D2296879
:102BD00021F0700101432960207800070AD560695F
:102BE000316801F07001884204D2316821F070012F
:102BF000014331602078C0060AD5A069316801F42C
:102C0000E061884204D2316821F4E061014331601F
:102C1000207880060CD5E1695846DBF8002002F0E8
:102C20007002914204D2026822F070020A430260EC
:102C300000F088F80E492A682B68C2F3032203F0DB
:102C40000F038A5CC95C02F01F0201F01F01D04033
:102C5000084A20FA01F11160074908600748006836
:102C6000BDE8F05FFFF730B9002000521844025869
:102C7000D060000818000024140000240C00002478
:102C800070B5144C3F220260124A24680832131DAA
:102C9000114D04F00704446016681C1D06F47066AC
:102CA0008660166806F00F06C660126802F07002B1
:102CB00002611A6802F0700242611A6802F4E0626E
:102CC0008261226802F07002C261286800F00F0081
:102CD000086070BD104402580020005230B500F06A
:102CE00031F80B4A0B490C4B15681468C5F30322E5
:102CF00004F00F048A5C095D02F01F0201F01F015D
:102D0000D040064A20FA01F119601060084630BD33
:102D100018440258D0600008180000241400002451
:102D200000B5FFF7DBFF05490968054AC1F3021149
:102D3000515C01F01F01C84000BD00001C44025856
:102D4000D0600008454970B545480968434B103BC1
:102D500011F0380208D00111082A03D0102A0BD034
:102D6000182A0BD0084670BD19688906FBD519686A
:102D7000C1F3C101C84070BD3A4870BD3749374DF5
:102D800018310C1D24350A68096826682D6802F080
:102D9000030406F00102C1F30511C5F3CC0515FBD0
:102DA00002F200EE102AB8EE400AE9B32F4ADFED36
:102DB0002E0AB7EE001A6CB1DFED2D1A012C01D0EE
:102DC000022C43D002EE101A1068F8EE422A81EE6F
:102DD000A22A1EE01C68A40611D51B6801EE901AF9
:102DE0001168C3F3C103F8EE612AD84001EE900ADE
:102DF000C1F30800F8EE611A81EEA22A0BE001EEA1
:102E0000901ADFED1C2A00BFF8EE611A106882EEFE
:102E1000A12AC0F3080001EE900AF8EE611A40EE14
:102E2000201A31EE810A00E015E022EE000A106857
:102E3000C0F34620401C00EE900AF8EE600A80EED7
:102E4000201ABCEEC10A10EE100A70BD01EE901AF5
:102E5000DFED092AD8E7002070BD000010440258B9
:102E60000090D00300366E01000000393044025853
:102E70000024744A0024744C001BB74B2DE9F05F0A
:102E800004007DD0FF4F2078FE4D1837DFF8F48323
:102E9000103DC00748D0D8F80000396800F038006D
:102EA000102815D0182803D101F0030002280FD0F4
:102EB0006068B0F5803F12D010B1B0F5A02F18D0E7
:102EC000286820F480302860286820F4802009E0F9
:102ED0002868800328D560680028D2D024E02868BC
:102EE00040F480302860606888B1FEF7B1FF064684
:102EF00009E0286840F480202860F0E7FEF7A8FF8A
:102F0000801B64287ED828688003F7D50CE0FEF784
:102F10009FFF064605E000BFFEF79AFF801B64286E
:102F2000F0D828688003F7D42078800756D5D8F8E1
:102F30000000DFF85093396810F03800A9F10C094F
:102F40000ED0182801D188070AD0E068A8B32968F4
:102F500021F0190101432960FEF77AFF064628E0B7
:102F60002868400702D5E06800288AD0E168286810
:102F700020F0190008432860FEF76AFF064606E0C5
:102F8000D2E000BFFEF764FF801B0228BAD8286891
:102F90004007F7D5217CD9F8002022F0FE4242EA12
:102FA0000161C9F8001019E0FEF752FF801B0228EA
:102FB000A8D828684007F7D5ECE7FFE7286820F095
:102FC00001002860FEF744FF064604E0FEF740FFDC
:102FD000801B022896D828684007F7D42078C006BE
:102FE00046D5D8F80000DFF89C92396800F0380028
:102FF000A9F10409082812D0182805D101F003000E
:10300000012800E0CEE00AD0E0690028286820D03E
:1030100040F080002860FEF71BFF064615E0286898
:10302000C00502D5E06980287ED194F82010D9F837
:10303000002022F07C5242EA0161C9F8001017E03A
:10304000FEF706FF801B0228A0D82868C005F7D528
:10305000EBE720F080002860FEF7FAFE064604E069
:10306000FEF7F6FE801B022890D82868C005F7D42A
:103070002078000729D5834861696430002981469A
:10308000016811D041F001010160FEF7E1FE064642
:1030900005E000BFFEF7DCFE801B022888D8D9F8C7
:1030A00000008007F6D510E021F001010160FEF775
:1030B000CFFE064605E000BFFEF7CAFE801B0228D1
:1030C00070D8D9F800008007F6D42078800623D580
:1030D000A0690028286810D040F480502860FEF7CE
:1030E000B7FE064605E000BFFEF7B2FE801B0228D1
:1030F00058D828688004F7D50EE020F48050286066
:10310000FEF7A6FE064604E0FEF7A2FE801B02289C
:1031100048D828688004F7D42078400751D5DFF8D4
:103120006891D9F8001000E015E141F48071C9F808
:103130000010FEF78DFE064605E000BFFEF788FE94
:10314000801B64282ED8D9F80000C005F6D54D4E56
:10315000A068603601280AD008B1052813D030686D
:1031600020F001003060306820F0040002E0306898
:1031700040F001003060A06841F2883A98B1FEF753
:1031800067FE81460AE0306840F004003060EEE7F8
:10319000FEF75EFEA0EB0901514503D830688007B9
:1031A000F6D50EE072E0FEF753FE814606E000BF62
:1031B000FEF74EFEA0EB0901514567D83068800745
:1031C000F6D4606A00287CD0DFF8B8A0D8F80010E8
:1031D0000AF1200A4FF6F87B0AF10408C1F3C20194
:1031E0000329AAF104096DD00228286820F0807014
:1031F000286003D0FEF72CFE044681E0FEF728FE8F
:10320000064604E0FEF724FE801B022875D82868D5
:103210008001F7D4E26A40F2F331386854F8283F6D
:10322000884340EA021018433860217B4FF4FE0CBB
:1032300022894FF0FE47208A4902267D521E401EF9
:10324000A1F5007189B2C2F308021143761E0CEA9F
:1032500000400143484607EA06621143CAF80010DD
:10326000D9F8001021F00101C9F80010D8F8003099
:10327000266A23EA0B0343EAC601C8F80010D9F80E
:10328000001004E0104402580048025835E0A269DA
:1032900021F00C011143C9F800100168E26921F026
:1032A000020111430160016841F48031016001684D
:1032B00041F400310160016841F48021016001683E
:1032C00001E06CE020E041F001010160286840F07D
:1032D00080702860FEF7BCFD044604E0FEF7B8FDF0
:1032E000001B022809D828688001F7D557E000BFE5
:1032F000FEF7AEFD001B022802D90320BDE8F09FB7
:1033000028688001F4D44AE039680128DAF800001E
:1033100021D0A26A01F0030393421CD1E26AC1F3F7
:1033200005118A4217D1216BC0F30802491E8A4257
:1033300011D1616BC0F34622491E91420BD1A16BA2
:10334000C0F30642491E914205D1E16BC0F306600D
:10335000491E814201D00120D0E7A16C4646D8F831
:103360000000C0F3CC00814219D0D9F800004D46CE
:1033700020F00100C9F80000FEF76AFD4FEA0007DF
:10338000FEF766FDB842FBD0A26C306820EA0B0065
:1033900040EAC2003060286840F001002860002048
:1033A000ACE770477047704710B5040003D094F83D
:1033B0003D0010B107E0012010BD002084F83C0062
:1033C000204600F022F8022084F83D002068211DEC
:1033D00000F048FC012084F8480084F83E0084F89E
:1033E0003F0084F8400084F8410084F8420084F8EB
:1033F000430084F8440084F8450084F8460084F8CB
:10340000470084F83D00002010BD704790F83D1043
:10341000012901D0012070471A4A022180F83D108D
:103420000168CB6843F00103CB60006890421AD07A
:10343000B0F1804F17D01449884214D01349884204
:1034400011D0134988420ED0124988420BD012493C
:10345000884208D01149884205D01149884202D0DB
:103460001049884207D181680F4A1140062906D0C9
:10347000B1F5803F03D0016841F0010101600020F7
:1034800070470000000001400004004000080040B8
:10349000000C0040000401400018004000400140C2
:1034A00000E0004000E400400700010070472DE903
:1034B000F041044600680027C6680569A90713D5CE
:1034C000B10711D5FA1E02610121217720688069B8
:1034D0008007204602D0FFF7E9FF04E000F08BF8F8
:1034E000204600F089F82777680716D5700714D5AD
:1034F000226802206FF00401116120772068806942
:1035000010F4407F204602D0FFF7D0FF04E000F027
:1035100072F8204600F070F82777280715D5300795
:1035200013D5226804206FF008011161207720680C
:10353000C0698007204602D0FFF7B8FF04E000F022
:103540005AF8204600F058F82777E80616D5F00616
:1035500014D5226808206FF01001116120772068CF
:10356000C06910F4407F204602D0FFF79FFF04E0BF
:1035700000F041F8204600F03FF82777E80708D030
:10358000F00706D021686FF001000861204600F0C6
:1035900034F8280601D4A80408D5300606D52168D9
:1035A0006FF4025008612046FFF7FCFEE80508D5DD
:1035B000300606D521686FF4807008612046FFF759
:1035C000F0FE680608D5700606D521686FF0400049
:1035D0000861204600F018F8A8060AD5B00608D5FC
:1035E00021686FF0200008612046BDE8F041FFF738
:1035F000DABEBDE8F081704770470068B0F1804FD7
:1036000001D1FEF72BBC70477047FEE71B48002135
:103610002DE9F041DFF860C00123C0F800C04FF091
:10362000030C0E270522C0E9021C03741225417405
:103630000824837404264261C0E9062702624262BC
:10364000C0E90A270263C0E90D13C0E91151C0E9BE
:1036500013614665C0E90F34C0E916418566C0E9CB
:103660001841FEF78BF8002803D0BDE8F041FDF7C4
:103670006FBBBDE8F081000000A00040B000002456
:103680001D4801212DE9F041DFF868C04FF4407E6C
:10369000C0F800C04FF0030C00230E27C0E902EC75
:1036A00001740522437440F23F3C81740425426159
:1036B0001226C0E90627C0E90821C0E90A2700F15F
:1036C0003C070263C0E90DC1082487E82A00C0E96D
:1036D0001246C0E91435C0E916438666C0E91843AE
:1036E000FEF74CF8002803D0BDE8F041FDF730BBF1
:1036F000BDE8F08100A40040500100241D480021D5
:103700002DE9F041DFF868C04FF4807EC0F800C0BA
:103710004FF0030C01240E25C0E902EC04740522CD
:10372000417404268474122742610823C0E90625E7
:10373000026240F27E6C4262C0E90A25C0E90E4195
:10374000C0E91016C0E91237C0E91416C0E91631F5
:103750008766C0E91831C0E90C2CFEF70FF8002885
:1037600003D0BDE8F041FDF7F3BABDE8F0810000F9
:1037700000D40040F0010024074A0021074810B59A
:1037800000F0D2FD0649074A08600021BDE810405C
:10379000054800F0C9BD000050600008C53A0008A7
:1037A00000000024E0600008453D000830B587B007
:1037B00014216846FCF7DDFE1E48016841F0040153
:1037C0000160016801F004010591016841F0800188
:1037D0000160016801F080010591016841F0080174
:1037E0000160016801F008010591016841F00101E3
:1037F0000160016801F001010591016841F00201D9
:10380000016000684FF460440B4D002200F002009C
:10381000214605902846FEF715FB00210094012063
:10382000CDE90101284603916946FEF7FDF907B08D
:1038300030BD0000E044025800080258FEE7FEE7F1
:1038400070B5AEB0B8216846FCF793FE002318248B
:1038500019464FF4004202208DE81C00C82506AB33
:10386000CDE903502026059083E84300020768460F
:103870001B920991FEF738FC002801D072B6FEE7D2
:103880002EB070BD2DE9F047454D044689464FF0F6
:10389000000A2868C04380070AD0414E283E30689D
:1038A00020F080603060FEF7D3FA0746B04608E0AB
:1038B0000120BDE8F08700BFFEF7CAFAC01B02284E
:1038C00067D8D8F800000001F6D4206829684FF4C2
:1038D000FE0721F47C313E0241EA00302860207A64
:1038E000A389B4F804C040022D4D2D495B1E227CF3
:1038F000ACF1010C1035091DA0F5007080B2521E0C
:10390000CCF3080C07EA034340EA0C00184306EA2C
:103910000262104328600868626920F0C00010430A
:1039200008600A68A06922F0200202430A60281D8C
:103930000A6822F010020A6002684FF6F873E46920
:103940009A4342EAC40202600868B9F1000F40F0ED
:1039500010020A6011D00868B9F1010F11D040F4CB
:1039600000100860D8F80000444640F08060C8F8B5
:103970000000FEF76DFA05460DE0086840F40020EF
:10398000EFE740F48010ECE7FEF762FA401B0228F4
:1039900001D903208DE720680001F5D5504688E75E
:1039A000284402582DE9F047454D044689464FF01A
:1039B000000A2868C04380070AD0414E283E30687C
:1039C00020F080503060FEF743FA0746B04608E02A
:1039D0000120BDE8F08700BFFEF73AFAC01B0228BD
:1039E00067D8D8F800008000F6D4208829684FF402
:1039F000FE0721F07C713E0241EA00502860207AE7
:103A0000A389B4F804C040022D4D2D495B1E227CD1
:103A1000ACF1010C1835091DA0F5007080B2521EE2
:103A2000CCF3080C07EA034340EA0C00184306EA0B
:103A30000262104328600868626920F44060104305
:103A400008600A68A06922F4007202430A60281D17
:103A50000A6822F480720A6002684FF6F873E4691B
:103A60009A4342EAC40202600868B9F1000F40F4C8
:103A700080720A6011D00868B9F1010F11D040F0CE
:103A800080700860D8F80000444640F08050C8F8C4
:103A90000000FEF7DDF905460DE0086840F48000FF
:103AA000EFE740F40000ECE7FEF7D2F9401B0228F4
:103AB00001D903208DE720688000F5D5504688E7BE
:103AC00028440258012000F08CFAFBE74FF0E02078
:103AD00010B5006902F0BCF8012803D0BDE8104021
:103AE00001F05ABC10BD000070B59CB04C21684676
:103AF000FCF73FFD202113A8FCF73BFD0220FEF759
:103B0000C9FA1E48016821F440410160016800249F
:103B100001F440411B9101688904FCD502200A9000
:103B200028230990C20301210D910425CDE900123B
:103B3000CDE90B030C261294CDE90E50CDE91064AB
:103B40006846FFF79BF908B172B6FEE740201A906D
:103B500008230501CDE9163013ABCDE918053F2147
:103B6000032283E8160013A81146FEF75BFF002826
:103B700001D072B6FEE71CB070BD000018480258B4
:103B80002D48F0B52D4A016841F4700101601068BC
:103B900000F00F00072804D2106820F00F00C01DAD
:103BA000106027490020264C10340B68254D43F047
:103BB00001030B6020600B682B400B60136803F05F
:103BC0000F03072B04D9136823F00F03DB1D1360C9
:103BD0001B4C1D4A18341D4B261D371D2060184CE8
:103BE0001B4D28343060261D3860371D23603B1D77
:103BF00035601C1D3A60251D2E1D1860331D226086
:103C00002860326018600B680D4A0D4C23F4802345
:103C1000D4320B60603420601068C0040BD4136889
:103C200043F2D2000B4943F48053136008601068DC
:103C300020F480501060F0BD88ED00E000200052BC
:103C4000004402587FEDF6EA800201010002020200
:103C50000000FF01004000520148FFF728BC0000AF
:103C6000900200242DE9F0472C4B4FF0804A2C4D58
:103C7000026898422B4E2C4F2C4C09D0504507D04F
:103C8000A84205D0B04203D0B84201D0A04205D12D
:103C9000D1F804C022F070024CEA0202DFF890C0B2
:103CA000DFF890809842DFF8909015D0504513D0FF
:103CB000A84211D0B0420FD0B8420DD0A0420BD0D4
:103CC000604509D0404507D0484505D01B4DA84266
:103CD00002D01B4DA84203D1CD6822F440722A4382
:103CE0008E684D6922F08002C6620E682A439842AF
:103CF000866207D0A04205D0604503D0404501D080
:103D0000484501D1096901630368012143F00403B7
:103D1000036041610260BDE8F087000000000140DF
:103D20000004004000080040000C00400004014076
:103D300000400140004401400048014000E00040D4
:103D400000E4004010B500F08DF90A4A00210A484D
:103D500000F0EAFA094C00220A21A060022000F0DB
:103D600003FA206200F0B0F900F0DCFABDE8104080
:103D700000F022BB04610008813D0008FC710024B2
:103D800088B000F05AF900EE100A9FED481B0020A1
:103D9000B8EE400B80EE012BBCEEC20B10EE107A99
:103DA00000F01FF900F042F9424C01220546510390
:103DB0002046FEF747F801222046D103FEF742F8DD
:103DC000FCF716FD40F20114082221460020FCF702
:103DD0001FFE661C082231460120FCF719FE40F246
:103DE0000319082249460220FCF712FEA0464FF0B4
:103DF000080A31A154463D4401ABD1E9000230A18B
:103E0000CDE90102D1E900212FA0CDE90321D0E9BC
:103E10000010CDE905109DF804009DF805209DF8DF
:103E2000061050409DF80D2048408DF80B009DF87D
:103E30000C009DF80E1050409DF8152048408DF85C
:103E400013009DF814009DF816105040424648405B
:103E50008DF81B000021CDF800A00846FCF77EFE7F
:103E6000002132460120009403ABFCF777FE0021CD
:103E70004A460220009405AB4C46FCF76FFE002337
:103E8000134A41461846FCF781FC114A00230120E1
:103E90003146FCF77BFC0E4A002302202146FCF74A
:103EA00075FC284600F0ABF8A3E700000000000016
:103EB0000000594000080258A1013412100000000F
:103EC000A102785620000000A1030001300000008C
:103ED000A8710024FEE7090700284FEA116104DBFE
:103EE00000F1E02080F80014704700F00F0000F1AE
:103EF000E02080F8141D70472DE9F041040006D041
:103F0000184E306884420AD10020BDE8F08150206C
:103F100080F31188BFF34F8FBFF36F8FFEE700F080
:103F20002DFF776B6569B66B00F048FFBD4201D08D
:103F3000B54201D10220E8E70B48854208D1A06ACA
:103F40000028F7D194F858000128F3D00320DCE7CB
:103F500005481438854202D00DB10120D5E7042070
:103F6000D3E700001C000024CC0700241FB5002468
:103F70000094019402940394FEF71AF801208DF83E
:103F80000C001F218DF8081087228DF809208DF86C
:103F90000D008DF8000068468DF80A408DF80E403F
:103FA0008DF8014001948DF80B408DF80F40FDF71E
:103FB000D1FF0420FEF70AF8FDF758FFFFF794FD44
:103FC000FFF73EFCFFF7F2FBFFF720FBFFF758FB84
:103FD000FFF794FB00F034F8FFF7CEFB00F058F841
:103FE000FEE710B5EFF3058111B16FF0050404E0B1
:103FF0004FF0000408B100F099FF204610BD38B51D
:104000000546EFF3058010B16FF005040CE00024C5
:1040100001F02CFE291A0090002903DD684600F00B
:10402000ABFF01E06FF00304204638BDEFF30580DD
:1040300008B101F021BE01F019BE4FF47A7070474B
:10404000EFF3058010B16FF0050070470449086870
:1040500010B14FF0FF30704701220A600020704716
:104060006C00002410B5EFF3058010B16FF005006F
:1040700010BD01F0EDFD20B1022804D04FF0FF305B
:1040800010BD012010BD01F0D3F8002010BD0000CC
:1040900010B5EFF3058010B16FF0050010BD0848B2
:1040A0000168012902D04FF0FF3010BD054A002100
:1040B00082F8141D0221016001F076F8002010BD85
:1040C0006C0000240BE000E070B5EFF3058010B148
:1040D0006FF0050413E001F0BBFD4FF0FF3510B1A8
:1040E00002280BD108E0012401F0E6FE012806D0E9
:1040F00001F0AEFD10B102E0002400E02C462046A5
:1041000070BD0000F8B56FF003021D466FF00206A7
:104110004FF00004EFF30583A3B1F0B1E9B1E5B9C5
:10412000002200926A4601F0CFFB012817D10098C7
:10413000B0B10C494FF080500860BFF34F8FBFF310
:104140006F8F0DE048B141B12A4601F01FFB0128F5
:1041500006D025B16FF0010402E0144600E03446B9
:104160002046F8BD04ED00E0F8B514464FF0000518
:10417000EFF3058212BB08B301B3A4B1D4E9023254
:1041800063B1502A1AD32269C2B100FB01F66769F4
:10419000B74213D3009501F04EF907E072B92269D6
:1041A00062B9626952B9002201F024F9050005D014
:1041B0000CB1216800E0002100F082FE2846F8BD25
:1041C000F8B56FF003021D466FF002064FF00004D1
:1041D000EFF30583ABB100B3F9B1F5B9002200925A
:1041E00013466A4601F054FA012818D10098B8B174
:1041F0000C494FF080500860BFF34F8FBFF36F8FB3
:104200000EE050B149B100232A4601F091F901288E
:1042100006D025B16FF0010402E0144600E03446F8
:104220002046F8BD04ED00E02DE9F0410D460146C1
:1042300021F001004FF0000401F00101EFF30582CD
:104240000AB1A41F16E048B1002929466FF0010603
:104250006FF0020708D001F043FC07E06FF00304A1
:1042600008E035B1344605E001F07CFB0128F8D1C7
:1042700000E03C462046BDE8F08170B505464FF0B1
:104280000004EFF3058050BB0DB1686800E000202A
:10429000C10701D0012600E0002600071FD46DB140
:1042A000D5E9021021B1502819D31EB1042002E033
:1042B00020B114E0012001F090F805E00EB10420D7
:1042C00000E0012001F07EF8040008D00DB129685B
:1042D00000E0002100F0F4FD0EB144F0010420469E
:1042E00070BD014670B521F001004FF0000401F0EF
:1042F0000101EFF305820AB1A41F11E028B16FF0AC
:10430000020529B101F023FA07E06FF0030407E08A
:1043100000231A46194601F00BF9012800D02C465B
:10432000204670BD01F08EBC2DE9FF414FEA01032C
:104330004FF00005EFF30581039561BB58B34FF0D3
:1043400080064FF018014FF000044AB3176807B118
:104350003C4697691FB139467F1E382F02D2177924
:10436000FF0703D0002004B0BDE8F081576907B112
:10437000BE08D2F808C0BCF1000F0DD0D5685C2D86
:1043800018D312693AB137B18DE80610324621468A
:1043900001F02DFC03900DE0D7685FB912694AB9AE
:1043A00003AACDE90012B2B2214601F0F3FB0128C5
:1043B00000D003950398D6E770B50546EFF3058066
:1043C00010B16FF005040FE04DB12846FFF794FDE2
:1043D000042807D00024284600F014FE04E06FF003
:1043E000030401E06FF00204204670BD2DE9F041A6
:1043F000134C0F460546E6682068001D00F060FC7F
:10440000681C07D137B12168BDE8F0410D48091D8E
:1044100000F0A8BC20683544B5424560216805D24B
:10442000A06B091DBDE8F04100F084BC606B091D64
:1044300000F080FCA06A854200D2A562BDE8F08150
:104440001C000024CC0700242DE9F041054600F0B3
:1044500095FC2D4C2D4FA068401CA060206810B129
:10446000606930B32BE02560A068012827D10026C1
:1044700006EB860007EB800000F04EFC761C382E21
:10448000F6D3234800F048FC2148143000F044FCE7
:104490001F48283000F040FC1D483C3000F03CFC38
:1044A0001B48503000F038FC194860631430A0639A
:1044B00005E0E86A2168C96A814200D82560606A1F
:1044C000401C60626864E86A2169884200D9206102
:1044D00000EB8000291D07EB800000F043FC00F09A
:1044E0006DFC606900280CD02068E96AC06A8842C7
:1044F00007D208494FF080500860BFF34F8FBFF3D9
:104500006F8FBDE8F08100001C0000241C03002414
:104510007C07002404ED00E038B500F02FFC104CBF
:104520002068C8B90F4800F0F7FB0E48143000F0BF
:10453000F3FB0C490020E16014312161A1F5827385
:104540000090A1F1B40210210A2000F074FF206055
:1045500010B105A100F0B4FCBDE8384000F02EBC5D
:1045600058000024D0080024546D7251000000004F
:1045700030B4026C0B46002A0BD0D0E90241114442
:10458000C160A14201D30168C160184630BCFBF78D
:1045900071BF30BC70472DE9F041856B1746026C46
:1045A0000446002682B1C7B1E068FBF763FFE1680B
:1045B000206C2268091AE160914202D2A168081AAF
:1045C000E060022F16D017E02068A8B9A06801F0BB
:1045D000BFFB06460020A0600EE06068FBF74AFFC4
:1045E000D4E90101226C10446060884204D3206841
:1045F000606001E005B16D1E6D1CA5633046BDE82D
:10460000F08110B5044690F8590058B101280CD03B
:1046100002280FD0502080F31188BFF34F8FBFF3D3
:104620006F8FFEE7206B00F0DDFB2046BDE81040F9
:1046300000F0D8BB10BD000011484FF4705110B508
:10464000420706D00E49C01D20F00700411AC1F5EF
:1046500070510C4C002301440839A4F1180221F0D8
:104660000701C4E900030C1A11604B600B60C0E93C
:10467000001494604FF000415460516110BD00007F
:10468000B00F002488000024144E4FF08058144CC2
:10469000DFF85090A6F29C4712E000BF00F06EFBDE
:1046A000F068C568281D00F00BFBA068401EA060E4
:1046B0006068401E606000F081FB2846FFF7A1FFA4
:1046C00060680028EAD138680128F9D9C9F8008063
:1046D000BFF34F8FBFF36F8FF2E70000B8070024DE
:1046E0001C00002404ED00E0002807D000218160B8
:1046F00001600B460A46C16000F01ABF7047000017
:1047000070B51D46049C51B1C4F80020C4E90F01E6
:104710000121204600F0C2FE84F84C5070BD246098
:10472000F4E72DE9F05F88469A4691001546DDE9E9
:104730000B940A9EA5228346206BFBF712FF206B89
:104740006FF0030101EB8501084420F007077807AB
:1047500007D0502080F31188BFF34F8FBFF36F8FC6
:10476000FEE7B8F1000F4FF000050ED00020221830
:1047700018F8001082F8341018F8001011B1401C1D
:104780001028F4D384F8435001E084F83450382ED4
:1047900000D33726E662201DC4E9136500F0C7FA8E
:1047A00004F1180000F0C3FA6565C6F13800A06195
:1047B00084F858505246246159463846646200F0E5
:1047C00067FAB9F1000F206001D0C9F80040BDE8D8
:1047D000F09F000030B5114900E011460A6882429E
:1047E000FBD34B685C18844203D1446808462344D9
:1047F0004B6043681D18954209D1084C183C246849
:10480000A24209D052681A4442600A6812680260E3
:10481000814200D0086030BD0460F9E788000024C0
:1048200070B50D4D914241604FF00004006106D813
:104830008169D21A8A4206D2011D286907E09A428C
:1048400003D2994201D3012403E0011DE86800F07E
:1048500071FA204670BD00005800002410B50446CF
:1048600000F08CFAA06B28B15FF0000400F0A6FA0B
:10487000204610BD0124F9E730B53C4D89B06BE00E
:104880000498002806DA059ADDE9060190470498A5
:10489000002861DB069C606910B1201D00F010FA51
:1048A00003A800F0D5F8024604980A2854D2DFE89D
:1048B00000F00505052D304705052D3094F828003A
:1048C00040F0010084F82800A06905990B460144D6
:1048D0002046FFF7A5FF50B3216A2046884794F889
:1048E0002800400738D50020009005980023A169D2
:1048F00042181946204601F071FBC0B9502080F3E0
:104900001188BFF34F8FBFF36F8FFEE794F8280035
:104910001EE094F8280040F0010084F82800059873
:10492000A06128B1811813462046FFF779FF13E0F4
:10493000502080F31188BFF34F8FBFF36F8FFEE7D6
:1049400094F82800810703D4204600F04BFA03E0D6
:1049500020F0010084F828002868002204A900F053
:1049600015FF00288CD109B030BD0000580000248C
:104970002DE9FC410F46054600F05AFC01A800F065
:1049800067F80446019818B101F096FABDE8FC8179
:10499000254EAFB130690068D0B300273068291BBD
:1049A0003A4600F0A1FA01F087FA0028EED11F493B
:1049B0004FF080500860BFF34F8FBFF36F8FE5E774
:1049C000A542EBD801F078FAF0682746C068C468C1
:1049D000201D00F075F994F82800410719D5A06949
:1049E0002B463A4641192046FFF71AFFA8B100208E
:1049F0002A46034601460090204601F0EFFA60B9CE
:104A0000502080F31188BFF34F8FBFF36F8FFEE705
:104A100007E020F0010084F82800216A204688473A
:104A2000B4E70127BAE700005800002404ED00E0D5
:104A30000648416B096829B1416BC968C968496872
:104A4000816270474FF0FF31FAE700001C0000243C
:104A500070B5054601F00AF9064E0446B068844276
:104A600003D200F009F8012000E000202860204671
:104A7000B46070BD58000024F8B5194D20E0C0683E
:104A8000C4680668201D00F01BF9216A204688478B
:104A900094F82800400713D5A0693044B04206D9E5
:104AA0002461211D6060E86800F044F908E00020FE
:104AB0003246034601460090204601F08FFA38B195
:104AC000E86801680029DAD12969C5E90310F8BD51
:104AD000502080F31188BFF34F8FBFF36F8FFEE735
:104AE0005800002408484068401C4FF0500080F3F4
:104AF000118804D0BFF34F8FBFF36F8FFEE7BFF372
:104B00004F8FBFF36F8FFEE790000024074CE068E3
:104B1000016841B1C0680021D0F80000FFF728FF0C
:104B2000FFF7AAFEF3E701210020F7E75800002471
:104B30002DE9F041044600F021F994F9455004F1C3
:104B4000240609E0606A48B1304601F07DF908B1F9
:104B500000F0A8FA6D1E6DB2002DF3DC4FF0FF36A9
:104B600084F8456000F02AF900F008F994F94450FF
:104B700004F1100709E0206948B1384601F064F9F2
:104B800008B100F08FFA6D1E6DB2002DF3DC84F8D1
:104B90004460BDE8F04100F011B900002DE9F0419A
:104BA0000027044600F044FB324E306808B9FFF796
:104BB00043FD706904424ED1C4B3083460070ED07F
:104BC00004F00700C0F108000444600707D050203B
:104BD00080F31188BFF34F8FBFF36F8FFEE72CB3C5
:104BE0007068844237D82348183001460D6801E0C8
:104BF00028460D466968A14202D229680029F7D1EA
:104C000031688D4227D007682968016008376868D5
:104C1000011B10290FD92819420708D0502080F312
:104C20001188BFF34F8FBFF36F8FFEE713E0416032
:104C30006C60FFF7CFFD69687068401A7060B268F9
:104C4000904200D2B060002072691143C5E90001B2
:104C5000F068401CF06001F02FF9780707D0502071
:104C600080F31188BFF34F8FBFF36F8FFEE7384695
:104C7000BDE8F081700000240449086818B1086894
:104C8000026D521C02650868704700001C00002479
:104C900070B5041F094E231F4FF0807521F00101EC
:104CA00025601C1F1960A0F120010B1F26604438ED
:104CB0000A606FF002051D6070BD0000E54A000843
:104CC000D0E9013201699A60D0E901235A604A684B
:104CD000824201D182684A60002202610868401E57
:104CE000086008687047000010B5044C8023046019
:104CF00004F15C000860136010BD0000F808002497
:104D000010B5044C4FF48073046004F15C0008603B
:104D1000136010BD540B00244FF0FF3300F1080165
:104D20000022C0E901130260C160016170470021E7
:104D30000161704730B50B685A1C02D000F10802BF
:104D400002E0026904E02246546825689D42FAD9CF
:104D500053684B6099608A60516008610168491C22
:104D6000016030BD42684A6093688B609368596007
:104D7000916008610168491C01607047502080F310
:104D80001188BFF34F8FBFF36F8F0A494868401CEB
:104D9000486001280CD10848006810F0FF0F07D0C8
:104DA000502080F31188BFF34F8FBFF36F8FFEE762
:104DB000704700009000002404ED00E008494868B6
:104DC00028B1401E486001D180F3118870475020FF
:104DD00080F31188BFF34F8FBFF36F8FFEE70000A2
:104DE0009000002470B500282AD0164DA0F10804C8
:104DF00061686869014207D1502080F31188BFF3D0
:104E00004F8FBFF36F8FFEE722683AB1502080F3D7
:104E10001188BFF34F8FBFF36F8FFEE7814361604F
:104E200000F006FA60686968084468602046FFF789
:104E3000D1FC2869401C2861BDE8704001F03CB8F5
:104E400070BD0000700000244FF0E02000210161DF
:104E50004FF47A728161072303490968B1FBF2F1CB
:104E6000491E4161036170471400002410B5FBF72F
:104E7000D9FA114910280ED300F1E0200A7890F8F1
:104E8000F003904207D2502080F31188BFF34F8F78
:104E9000BFF36F8FFEE709488968006800F4E0609F
:104EA000884207D9502080F31188BFF34F8FBFF39A
:104EB0006F8FFEE710BD0000900000240CED00E0B5
:104EC000084B5FF0000210B553F832401CB1521C81
:104ED000082AF9D310BD03EBC20443F83210606016
:104EE00010BD0000DC02002470B515460E460446D5
:104EF000FFF744FF94F944100020491C01D184F8C5
:104F0000440094F94510491C01D184F84500FFF78D
:104F100055FFA06B28B904F124002A46314600F061
:104F2000DFF82046BDE87040FFF702BE020010B572
:104F300014D00F48006B38B1502080F31188BFF3B4
:104F40004F8FBFF36F8FFEE700F072F9002110461C
:104F5000FFF74CFA00F0B0FF002807D105494FF0E9
:104F600080500860BFF34F8FBFF36F8F10BD0000FC
:104F70001C00002404ED00E070B504000D460BD0C9
:104F800095B11E4A106BB8B1502080F31188BFF361
:104F90004F8FBFF36F8FFEE7502080F31188BFF370
:104FA0004F8FBFF36F8FFEE7502080F31188BFF360
:104FB0004F8FBFF36F8FFEE700F03AF92368D26896
:104FC0005919934204D98B420AD9914202D807E079
:104FD0008B42FAD9881A21600021FFF707FA00E016
:104FE000216000F069FF002807D105494FF080508B
:104FF0000860BFF34F8FBFF36F8F70BD1C0000249C
:1050000004ED00E070B50546FFF7B8FE1E4C05B98B
:105010002568281DFFF754FEA86A18B105F118008D
:10502000FFF74EFE606A401C60622068854207D12F
:105030001648291DFFF796FE6068401C606007E077
:10504000A068401EA0602846FFF7DBFAFFF7F0FCDF
:10505000FFF7B4FE6069002814D02068854211D1A2
:10506000206B38B1502080F31188BFF34F8FBFF30E
:105070006F8FFEE706494FF080500860BFF34F8FF7
:10508000BFF36F8F70BD00001C000024B807002420
:1050900004ED00E002490A6A0260C9684160704795
:1050A0001C00002401490120C86170471C00002435
:1050B00010B50C4650B1094909681831FFF73AFE9E
:1050C0002046BDE810400121FFF790B9502080F341
:1050D0001188BFF34F8FBFF36F8FFEE71C000024D2
:1050E00070B514460D4668B10A4909681831FFF7D2
:1050F00039FE0CB14FF0FF3521462846BDE870401F
:10510000FFF774B9502080F31188BFF34F8FBFF3BE
:105110006F8FFEE71C00002470B5002804463ED0C7
:10512000226DA2B1E06C884200D30146E06A884259
:1051300035D0012A33D11A4D2A6894420FD150201C
:1051400080F31188BFF34F8FBFF36F8FFEE75020BE
:1051500080F31188BFF34F8FBFF36F8FFEE7A26913
:10516000E162002A02DBC1F13801A1610D4E00EBC2
:105170008000616906EB8000814210D1201DFFF79D
:105180009FFDE06A2969884200D9286100EB800010
:10519000211D06EB8000BDE87040FFF7E3BD70BD48
:1051A0001C0000241C03002430B587B0002405AA8D
:1051B00004A9039403A80494FFF796FDDDE9030115
:1051C00000940023CDE90110174815A1059A00F0BD
:1051D0000EFD164D0028E8621FD000F0CFFE01281A
:1051E00009D0401C19D1502080F31188BFF34F8F94
:1051F000BFF36F8FFEE7502080F31188BFF34F8F0E
:10520000BFF36F8F01214FF0FF30A8626961EC603E
:1052100007B0BDE8304000F045B807B030BD000031
:1052200049444C4500000000894600081C00002449
:105230000248016B491C0163704700001C000024F8
:10524000164810B5016B11B10121C16110BD0021DB
:10525000C161134A016901E0B9B1491E01EB810343
:1052600052F82330002BF7D001EB810302EB8302CD
:1052700002F1080453685B685360A34201D15B6884
:105280005360DA680260016110BD502080F311881C
:10529000BFF34F8FBFF36F8FFEE700001C000024A9
:1052A0001C03002437481CB5374902688A4207D1DD
:1052B000502080F31188BFF34F8FBFF36F8FFEE74D
:1052C00031490068491E884207D1502080F3118877
:1052D000BFF34F8FBFF36F8FFEE72C49FF200A7893
:1052E0000192087008788DF800009DF800209DF864
:1052F000000002F0F002824207D0502080F31188B3
:10530000BFF34F8FBFF36F8FFEE79DF8002007209C
:105310001F4C02F050022270A06005E09DF80020B2
:1053200052008DF80020401E9DF800201206F5D492
:105330000328A06007D0502080F31188BFF34F8F5F
:10534000BFF36F8FFEE74FF44070A06001980870C4
:105350000C482030016841F470010160016841F09F
:1053600070410160FFF770FD00206060FBF722F8DC
:105370000848016841F040410160FBF707F8002050
:105380001CBD000000ED00E071C20F4100E400E030
:105390009000002434EF00E0502010B580F3118815
:1053A000BFF34F8FBFF36F8F00F06EFC18B104494D
:1053B0004FF080500860002080F3118810BD00007D
:1053C00004ED00E000210246012010B500F012F8C3
:1053D0000446FFF789F9204610BD38B500220B4678
:1053E00011460090012000F026F80446FFF77CF9F2
:1053F000204638BDF8B5050017460E4613D005FB0C
:1054000006F05030FFF7CAFB04000AD0002084F8F1
:10541000460004F150023B46314628460094FFF70F
:105420006FF92046F8BD502080F31188BFF34F8FED
:10543000BFF36F8FFEE7F8B5069D18B153B1CAB13F
:1054400081B120E0502080F31188BFF34F8FBFF36C
:105450006F8FFEE7502080F31188BFF34F8FBFF3AB
:105460006F8FFEE7502080F31188BFF34F8FBFF39B
:105470006F8FFEE739B1502080F31188BFF34F8F53
:10548000BFF36F8FFEE750241C46012683F8466069
:1054900000932B46FFF734F92046F8BD2DE9F0477D
:1054A00004008A4629D0FFF769FC21680025D4E969
:1054B0000F23D4F840C004F1100810460E46401ED9
:1054C0004FF0FF3902FB031200FB0C10BAF1000F82
:1054D000A563666084F8449084F84590C4E902208E
:1054E00013D04046FFF718FC04F12400FFF714FC2A
:1054F000FFF764FC0120BDE8F087502080F311889D
:10550000BFF34F8FBFF36F8FFEE720690028EFD006
:10551000404600F099FC0028EAD004494FF0805042
:105520000860BFF34F8FBFF36F8FE1E704ED00E03A
:105530002DE9FF4704001D4682B08A464FF000085F
:1055400003D0BAF1000F08D011E0502080F3118889
:10555000BFF34F8FBFF36F8FFEE7206C38B1502041
:1055600080F31188BFF34F8FBFF36F8FFEE7022DDB
:105570000AD1E06B012807D0502080F31188BFF3D7
:105580004F8FBFF36F8FFEE700F062FB3F4F4FF08E
:1055900080564FF0000948B9049838B1502080F384
:1055A0001188BFF34F8FBFF36F8FFEE7FFF7E6FB66
:1055B000A06BE16B884207D3022D05D00498D0B1CF
:1055C000B8F1000F1AD01EE02A4651462046FEF7D9
:1055D000E2FF616A19B104F1240000F035FC20B14A
:1055E0003E60BFF34F8FBFF36F8FFFF7E7FB0120E4
:1055F00006B0BDE8F087FFF7E1FB22E06846FFF761
:1056000049FD4FF00108FFF7D9FBFFF711FEFFF747
:10561000B5FB94F94400401C01D184F8449094F9FE
:105620004500401C01D184F84590FFF7C7FB04A951
:10563000684600F073FA30B12046FFF779FA00F0BF
:105640003BFC0020D4E7FFF799FBA06BE16B88429D
:1056500013D1FFF7B3FB049904F11000FFF728FD05
:105660002046FFF765FA00F027FC00289ED13E6037
:10567000BFF34F8FBFF36F8F98E7FFF79FFB204675
:10568000FFF756FA00F018FC90E7000004ED00E088
:105690002DE9F04704001F469046894603D0B9F132
:1056A000000F08D011E0502080F31188BFF34F8F16
:1056B000BFF36F8FFEE7206C38B1502080F3118864
:1056C000BFF34F8FBFF36F8FFEE7022F0AD1E06B5E
:1056D000012807D0502080F31188BFF34F8FBFF30C
:1056E0006F8FFEE7FFF7C2FB5020EFF3118680F3C8
:1056F0001188BFF34F8FBFF36F8FA06BE16B8842B0
:1057000006D3022F04D0002086F31188BDE8F0876D
:1057100094F94550A06B3A4649462046FEF73BFFB8
:10572000681C04D06D1C84F845500120ECE7606AC9
:105730000028FAD004F1240000F086FB0028F4D001
:10574000B8F1000FF1D00121C8F80010EDE710B555
:10575000040009D000F076FAA168884214D1E0680C
:10576000401EE06008D00DE0502080F31188BFF3A8
:105770004F8FBFF36F8FFEE7002320461A4619466E
:10578000FFF7D6FE012010BD002010BD2DE9F74720
:1057900004008A4683B04FF0000603D0BAF1000F30
:1057A00008D011E0502080F31188BFF34F8FBFF372
:1057B0006F8FFEE7206C38B1502080F31188BFF363
:1057C0004F8FBFF36F8FFEE700F042FADFF8F480EF
:1057D0004FF080574FF0000948B9059838B1502074
:1057E00080F31188BFF34F8FBFF36F8FFEE7FFF792
:1057F000C5FAA56BC5B151462046FEF7B9FE6D1E30
:10580000A563206950B104F1100000F01DFB28B120
:10581000C8F80070BFF34F8FBFF36F8FFFF7CEFA5A
:10582000012006B0BDE8F087059808B11EB106E07A
:10583000FFF7C4FA27E06846FFF72CFC0126FFF7C4
:10584000BDFAFFF7F5FCFFF799FA94F94400401C04
:1058500001D184F8449094F94500401C01D184F8AA
:105860004590FFF7ABFA05A9684600F057F9002804
:1058700020460AD0FFF75CF900F01EFB2046FEF739
:10588000EDFF0028B3D00020CBE7FEF7E7FF90B193
:10589000059904F12400FFF70BFC2046FFF748F9B7
:1058A00000F00AFB0028A2D1C8F80070BFF34F8FA8
:1058B000BFF36F8F9BE72046FFF73AF900F0FCFA41
:1058C00095E7000004ED00E02DE9F0470400904664
:1058D000894603D0B9F1000F08D011E0502080F3C1
:1058E0001188BFF34F8FBFF36F8FFEE7206C38B185
:1058F000502080F31188BFF34F8FBFF36F8FFEE707
:10590000FFF7B4FA5020EFF3118680F31188BFF34C
:105910004F8FBFF36F8FA76BFFB194F94450494687
:105920002046FEF725FE681CA7F10107A76304D0F7
:105930006D1C84F84450012010E020690028FAD042
:1059400004F1100000F080FA0028F4D0B8F1000F44
:10595000F1D00121C8F80010EDE7002086F311888E
:10596000BDE8F0872DE9F3434FF00006040035460B
:1059700083B009D0206C78B1502080F31188BFF338
:105980004F8FBFF36F8FFEE7502080F31188BFF376
:105990004F8FBFF36F8FFEE700F05AF9DFF83C81BD
:1059A0004FF080574FF0000948B9049838B15020A3
:1059B00080F31188BFF34F8FBFF36F8FFEE7FFF7C0
:1059C000DDF9A06BC8B12168401EA06311B9FFF7D3
:1059D00053F9A060206950B104F1100000F034FACE
:1059E00028B1C8F80070BFF34F8FBFF36F8FFFF778
:1059F000E5F9012005B0BDE8F083049808B166B16F
:105A00000FE03DB1502080F31188BFF34F8FBFF3FB
:105A10006F8FFEE7FFF7D2F95EE06846FFF73AFBCB
:105A20000126FFF7CBF9FFF703FCFFF7A7F994F97D
:105A30004400401C01D184F8449094F94500401C76
:105A400001D184F84590FFF7B9F904A9684600F040
:105A500065F80028204612D0FFF76AF800F02CFA0B
:105A60002046FEF7FBFE0028A9D075B3FFF786F9A4
:105A7000606A58B3206B0068C0F1380128E0FEF777
:105A8000EDFEE0B1206838B9FFF778F9A06800F0C2
:105A90009DF90546FFF792F9049904F12400FFF7F8
:105AA00007FB2046FFF744F800F006FA002886D1ED
:105AB000C8F80070BFF34F8FBFF36F8F7FE72046AA
:105AC000FFF736F800F0F8F979E705E0FFE7002185
:105AD000A068FFF721FB9DE700208BE704ED00E0C5
:105AE00070B504000D4607D000F0ACF8A1688842FC
:105AF0000AD1E16801200EE0502080F31188BFF345
:105B00004F8FBFF36F8FFEE729462046FFF72AFF2E
:105B1000002802D0E168491CE16070BD2DE9F04128
:105B200005000C4612D0CCB1FFF728F9184E2068BA
:105B3000F268471C6B68A2EB030117D02F68366A26
:105B4000B74215D0934213D801251CE0502080F3B2
:105B50001188BFF34F8FBFF36F8FFEE7502080F3A4
:105B60001188BFF34F8FBFF36F8FFEE700250AE068
:105B7000884205D9401A20602846FFF78BFAF5E7DE
:105B8000002020600125FFF719F92846BDE8F081C3
:105B90001C0000242DE9FF5F994616468A4683467D
:105BA0009000DDE90E87FEF7F9FF05001CD05C20B0
:105BB000FEF7F4FF040014D00020256384F8590098
:105BC0004B46CDE90087CDE9024032465146584662
:105BD000FEF7A7FD2046FEF737FC012004B0BDE824
:105BE000F09F2846FFF7FEF84FF0FF30F6E7F0B5DC
:105BF00085B0DDE90B740A9DA7B1DCB15C26276393
:105C0000022684F85960002703970DF1100C0095C7
:105C1000CDE901C4FEF785FD2046FEF715FC04988A
:105C200005B0F0BD502080F31188BFF34F8FBFF354
:105C30006F8FFEE7502080F31188BFF34F8FBFF3C3
:105C40006F8FFEE701480068704700001C000024C9
:105C50000548416919B1006B18B100207047012057
:105C600070470220704700001C0000240148C068F3
:105C7000704700001C00002410B5FFF7F7F801483A
:105C8000C06810BD1C0000242DE9F0412E4C206B93
:105C9000002728B1A069401CA0613846BDE8F0810A
:105CA000E668761CE66013D1606B006838B150205E
:105CB00080F31188BFF34F8FBFF36F8FFEE7606BE8
:105CC000A16B6163A063206A401C2062FEF7B0FEF6
:105CD000DFF87880A06A864209D3606B0068A0B1C3
:105CE000606BC068C5686868864211D2A06220688F
:105CF000C06A00EB800158F82100012800D9012773
:105D0000E0690028C9D00127C7E74FF0FF30EDE771
:105D1000281DFEF7D5FFA86A18B105F11800FEF797
:105D2000CFFFE86A2169884200D9206100EB800139
:105D300008EB8100291DFFF715F82068E96AC06AA1
:105D40008142CAD30127C8E71C0000241C03002499
:105D500070B504464FF0000190B31A4D2868844294
:105D600007D0502080F31188BFF34F8FBFF36F8FA0
:105D7000FEE7206D38B1E36C401EE26A20659A426E
:105D80001ED040B11CE0502080F31188BFF34F8F2C
:105D9000BFF36F8FFEE7201DFEF792FFE06CC0F1AE
:105DA0003801A161E0622969884200D9286100EBCD
:105DB0008000054901EB8000211DFEF7D3FF012182
:105DC000084670BD1C0000241C03002470B5002888
:105DD00004464FF000002BD0194DE16A2A68D26AC0
:105DE000914226D2A069002804DB2868C06AC0F16D
:105DF0003800A061134E01EB8101606906EB81015F
:105E0000884211D1201DFEF75BFF2868C06AE0625E
:105E10002969884200D9286100EB8000211D06EB2A
:105E20008000FEF79FFF02E02868C06AE062012060
:105E300070BD2968E26CC96A8A42F8D370BD00005F
:105E40001C0000241C03002470B5C068C46854B151
:105E500004F118000646FEF733FF144D286B50B1CD
:105E60001348314615E0502080F31188BFF34F8F5F
:105E7000BFF36F8FFEE7201DFEF722FFE06A29695E
:105E8000884200D9286100EB80000A4901EB8000BC
:105E9000211DFEF767FFE06A2968C96A884203D9B5
:105EA0000121E961084670BD002070BD1C0000247E
:105EB000A40700241C0300242DE9F0472C4D286B77
:105EC0000024274638B1FEF759FF286B401E28638F
:105ED000286B40B147E0502080F31188BFF34F8F0B
:105EE000BFF36F8FFEE7234E0120A968D9B3A6F553
:105EF000916980463068E0B1F068C46804F1180028
:105F0000FEF7DEFE201DFEF7DBFEE06A296988420F
:105F100000D9286100EB800109EB8100211DFEF70B
:105F200021FFE06A2968C96A8842E3D3C5F81C806A
:105F3000E0E70CB1FEF77CFDAC694CB14FEA080616
:105F4000FFF7A2FE00B1EE61641EF9D10020A86146
:105F5000E86940B1084901274FF080500860BFF35D
:105F60004F8FBFF36F8FFEF729FF3846BDE8F087EC
:105F70001C000024A407002404ED00E010B586B046
:105F8000FEF7CAFA114C2068B8B10020039005AAA8
:105F9000049004A903A8FEF7B3FEDDE90321022063
:105FA00000238DE807000C4809A1059AFFF71FFEA2
:105FB000606010B106B0012010BD502080F3118840
:105FC000BFF34F8FBFF36F8FFEE700005800002430
:105FD000546D7220537663000D4B00082DE9FF418C
:105FE0001E46134602004FF000000A9D16D0144CC6
:105FF0002768002F0FD006290292CDE9001317DA87
:10600000FFF726FE02284FF000030FD00022206881
:106010006946FFF78DFA04B0BDE8F081502080F3A7
:106020001188BFF34F8FBFF36F8FFEE72A46EEE76D
:106030000023324669463846FFF72AFBEBE70000AB
:10604000580000244FF04070E1EE100A7047000045
:1060500028610008000000000000000000000000AF
:106060000000000000020000180000000000000016
:10607000000000000001020304050607080C1014CC
:106080001820304000000000000000000000000068
:1060900000000000000000000100000002000000FD
:1060A00003000000040000000000000005000000E4
:1060B00000000000000000000000000006000000DA
:1060C00000000000000000000000000007000000C9
:1060D000000000000102030401020304060708098E
:1060E0003461000800000000000000000000000013
:1060F000000000000004000030000000000000006C
:1061000000000000406100080000000000000000E6
:106110000000000000000000000400001800000063
:10612000000000000000000064656661756C745436
:1061300061736B005461736B5F496E69740000009A
:10614000626C696E6B00000068610008000000244A
:10615000B00000000803000818620008B000002426
:1061600068A20000240300080000000000000000F6
:106170000100000010000000000000000090D003AB
:106180000090D003000000000000000000000000AC
:1061900000000000000000000000000000000000FF
:1061A00000000000000000000000000000000000EF
:1061B00000000000000000000000000000000000DF
:1061C00000000000000000000000000000000000CF
:1061D00000000000000000000000000000000000BF
:1061E00000000000000000000000000000000000AF
:1061F000000000000000000000000000AAAAAAAAF7
:10620000000000000000000000000000000000008E
:08621000000000000000000086
:04000005080002CD20
:00000001FF
